:020000000B28CB
:10000800DE0003088312A0000A08A1009E288316B8
:10001800FF2390008301352900308A000408840AF0
:100028008207003400340F341E342D343C344B34F2
:100038005A346934783487349634A534B434C334A4
:10004800D234E134F034FF348312A5001230250293
:1000580003183628AA012508013E84001020A900AB
:10006800FF30A800123025022430031C492825023D
:1000780003184828AA01FF30A9002430A400250845
:10008800240284001020A800243025023630031CE6
:1000980059282502031858282508DD3E8400102019
:1000A800AA00FF30A900A801363025024830031CF9
:1000B8006B28250203186A28FF30AA004830A400DC
:1000C8002508240284001020A900A8014830250230
:1000D8005A30031C7B28250203187A28FF30AA000F
:1000E800A9012508B93E84001020A8005A3025022D
:1000F800031C8C286C30250203188C286C30A40053
:100108002508240284001020AA00A901FF30A800B5
:1001180025086C3A031D9328A801A901AA012508FE
:100128006D3A031D9B28FF30A800A900AA002508E6
:10013800AB00080001300B1D00398B1E0039003858
:100148000319C5280B11D7308100AC0A2B086C3A6B
:100158000319C228AC08031DB42885168514051494
:100168002C082A06031985122C082906031985105C
:100178002C082806031DC5280510C528051085105C
:10018800851201300B1C00398B1D0039003803190A
:10019800EB28003005190130A3000030051A0130A2
:1001A800A2000B1000302F18013023060319E8288D
:1001B80023030319E82822030319E528AE01AE0A30
:1001C800E628AE01AD01AD0A2F1023182F148312B3
:1001D80021088A0020088300DE0E5E0E09001A211D
:1001E8006C302820851910292B086C3A031DFE282D
:1001F8006D30FF286C302820851D0029FF30A600AF
:10020800A7010130A6020030031CA703A702260A93
:100218000319270A031D05292D0BF628AD012E0306
:10022800031D18293F21F6284821F6288B0107309D
:10023800990083169F011C3085008312850183165F
:10024800811315151516161616158B150B100B1789
:10025800811281150111811001108B160B118B175A
:100268000800AF01A801A901AA01AB01AC01AD01C9
:10027800AE018301F328AB03FB302B02031C462994
:100288006B30AB002B082828AB0A6C302B02031804
:06029800AB012B08282831
:02400E00C43FAD
:10420000540049004D004F00460045005900200071
:104210004E004F0053004F005600200020002000A9
:104220005700570057002E002000200020002000DB
:104230004C00410042004B00490054002E00200079
:104240005200550020002000200020002000200007
:00000001FF
